S11300C100FF01FF010001010001FF01FF00FFFF2B
S11300D12E2A4B420620039C08D7098E06010C14D4
S11300E1037C03700AAF0A877EE07E7EE06B7EE0CC
S11000F1677EE0CC7EE1D17EE1AC7EA04ACA
S11301008EA042CE0C55BD04AECE00204FA70008F1
S11301108C00C126F7CE0C68BD04AEBD00F8815337
S113012027037C0055CE0071C640BD00FB81FC2333
S1130130048604201981F723048603201181E02317
S1130140048602200981A02304860120014F7F0038
S1130150567D005527169756BD00FB81F023048673
S113016003200981C02304860220014F9B56A70067
S11301709B549754BD00FB8438AA00A700085A2753
S1130180037E012ABD00FB840716BD00FB8407978C
S113019021D7227C0020CE0071BD04D48640AA0061
S11301A0A7008D26BD00FB8B00199738BD00FB848A
S11301B07F8A108B001997378D2F7D0055270716DE
S11301C08D2780001B199739202A7F005786309786
S11301D058973C7F00597F003D860F9746CE0061BB
S11301E06F00088C006726F839BD00FB840F8A2253
S11301F08B001939BD00FB84079747BD00FB8407BA
S11302009748BD04BECE0C76BD04AE96218D4EBD7E
S113021002AD96228D47CE0E53BD04AECE006DC600
S113022003BD00F8A700085A26F7CE0C98BD04AE0B
S11302308D30CE0CA1BD04AE8D39CE0CACBD04AE58
S11302407F003196399732BD0345CE0CB4BD04AE60
S11302508D47CE0CBFBD04AE8D497E02BB8B317E73
S113026000F5DE37DF31BD0345862EBD00F5962847
S11302707E00EC96547F00317F0032C60A10250CB4
S11302807C0032D13226F67C003120EC1BD6325869
S11302905858581B97327E034596478DC08D0E964D
S11302A04820BA96498DB68D04964A20B0862D7E94
S11302B000F5DF319B329732DE31399639913B229A
S11302C0037E0B4C7D005426037E0B517D00672773
S11302D009CE0FA4BD04AE7E0A9DBD0B7A860291A1
S11302E04E27487F004E7D002627034A974EBD00C7
S11302F0FB81FC230DCE0EF3BD04AE860297667E11
S11303000370BD00FB81FC23037E0BB0BD0AFA7DA4
S113031000582A037E0B44860391582302974E7D8E
S1130320003C2A074F9757973C973DCE0CC8BD0415
S1130330AE7F00297F0070BD086348CE00D5BD02A2
S1130340B2EE006E007F004D9631271184F0270530
S11303509631BD00EF9631BD00EC7C004D96327DA8
S1130360004D260484F02703BD00EF96327E00EC96
S11303707F0057CE0CD3BD04AE7E02BB963C8101F8
S113038023F77D006626E97C0057CE003C86029761
S1130390317F0032BD08BBCE0CE120DA7D0062273C
S11303A0037E0C0BBD04B37F0050964E81022603DE
S11303B0BD01CACE00B1DF33BD0457CE0D4CBD0024
S11303C0E9BD0262BD0457CE0D57BD00E9964E2724
S11303D01A8101271181032705CE0C812003CE0D3C
S11303E061BD00E9200ACE0D6820F6CE0D6C20F127
S11303F08D65CE0D72BD00E9BD02998D5ACE0D7D7D
S1130400BD00E9BD02A38D4FCE0D88BD00E9DE58C5
S1130410DF31BD03458D40CE0D93BD00E9BD0273B0
S11304208D35CE0DA0BD00E9DE3CDF31BD03457D39
S113043000572705CE0C722003CE0C88BD00E98D31
S113044016CE0DAABD00E97F003196468B001997A0
S113045032BD03457E02BBBD04B3860297307F00E4
S11304604F86049751DE33A6009756964A9150263C
S11304700D9649914F26078645BD00F5200F9656E7
S1130480CE00D18403BD02B2A600BD00F5BD00F2CA
S1130490DE337C004F7A005127069656444420C927
S11304A008DF33A6007A003026B77C0050398D036C
S11304B07E00E9DF35CE0DB6BD00E9DE35397F00BB
S11304C026CE00B1C6104FA700085A26FACE0071F6
S11304D09647D64897565D27098608084A26FC5A47
S11304E026F796562704084A26FC7D002027047F19
S11304F0002039DF6BE600D7522736C407270AD716
S113050030D726860297538D62D652C438270B54AF
S11305105454D730860197538D51D652C540270A7B
S113052086019730860397538D41D6522A037C0067
S113053067BD00FB8407974BBD00FB8407974CBD48
S113054005B37D004D26EA964B9749964C974AD6BB
S11305502658CE003E6F006F01BD00FB8B00197F53
S113056000319732BD08B85A26EF39CE00B1BD002C
S1130570FB840F975ABD02B2E600BD00FB840397CB
S113058056270556564A26FBC50326DFDA539656E8
S1130590270559594A26FBE7007A003026CD9653A1
S11305A08103260ED65A0C56965624028B049723A2
S11305B0D724397F004DDF35CE00B1964C2705088E
S11305C0084A26FB964B81032303088004E6009720
S11305D056270554544A26FBC4032710D74D7D00E3
S11305E02927097D00702607C1022703DE3539C695
S11305F0FC965627060D59594A26FBE400E70020CD
S1130600EB7D006527037E0C0B7D004626037E08E8
S11306105A7C0070BD00FB840F8A04972D7A004633
S11306207F002A7F0025CE0CECBD04AEBD0863819B
S1130630072234972C7D00702622CE0CF5BD04AE23
S1130640BD0863972D7D002B2609972A7D0061261E
S1130650B52000BD00F8810D26F9962CCE00C148C6
S1130660BD02B2962D26037E02BB97307D002A2759
S113067004860F97309649D64AAB00EB01BD083685
S11306807D002E27037E070D7D002F27037E070D97
S1130690974BD74C7D00702705BD04B38D1F7C009C
S11306A029BD05B3964D272B7D007027037E07EFE8
S11306B0810226037E0799CE0D03BD04AE964BBD81
S11306C0025DBD02AD964CBD025D7D00702701390F
S11306D07E075A7D0070270C964BD64C7A00302644
S11306E0987E082D964B9749964C974ABD00FB81FE
S11306F080230A8601BD08808603BD08A87A0030DD
S113070027037E06757D002A26037E075A7D007026
S113071027037E082D962D97309647D6487D002ACC
S11307202760AB00EB01974BD74CBD08367D002EFC
S113073027037E07CC7D002F27037E07CC964B979B
S113074047964C97487C00258606BD08808630BDB8
S113075008A87A003026C2BD04BE7F004E962191BF
S113076047261CD622D14826169623D6244C9049D7
S11307708102220B5CD04AC10222048602974E7E7B
S113078002BB9B2EDB2F81072242C107223E9747E3
S1130790D7488607BD088020BECE0D10BD04AE86A6
S11307A00197307F002A7C005B7A00547A00267C13
S11307B00070BD06BDCE0FC0BD04AEC66ABD0BE958
S11307C0CE0E60BD04AEBD02737E06E4CE0D24BD24
S11307D004AE96604C81032609CE0F13BD04AE7E91
S11307E00B5997607D002526037E075A7E0757CE56
S11307F00D31BD04AE964D8102261A7A00267A0088
S1130800547C005BCE0E4BBD00E9CE0E60BD04AE41
S1130810BD0273200D8101260C7C005CCE0E41BD0F
S113082000E97E02BBCE0E467C005D20F2CE0D3E7A
S1130830BD04AE7E075A7F002E7F002F4D2A057A15
S1130840002E2007810723037C002E5D2A047A00F2
S11308502F39C10723037C002F39CE0C8CBD04AE85
S11308607E02BB4F972BBD00F8812E27F7813922DA
S113087007812F2303803039CE0E3DBD00E920E3EC
S11308809B288109231F800A97287F0031860197BE
S113089032DF35CE0037BD08B8CE003ABD08B8BD4A
S11308A00BA0DE3539972839DF35CE00587F00316B
S11308B09732BD08BBDE35390C200D8699903197EF
S11308C0318699903297320DA601993219A701A663
S11308D000993119A700397D006327037E0C0B7F33
S11308E000427F00437F00447F0045CE0DBDBD0420
S11308F0AEBD0299BD04B3BD04B3964726037C0084
S113090044810726037C0045964826037C004281E7
S11309100726037C0043DE6B86F7BD02B27D0042EE
S113092027048D5B20028D1A8605BD02B28D1386C5
S113093005BD02B27D004327048D4420028D037E51
S113094002BBA6007D004427014F8D11A6008D0D2A
S1130950A6007D004527014F8D037E04B3168480D5
S11309600C4949BD00EC1784404444BD00EF178492
S11309703848BD00EF178407BD00EC087E00F286FE
S11309800397304F8DD77A003026F87E04B37D006C
S11309906427037E0C0B7D00572705CE0DC9202745
S11309A0CE0DDCBD04AEDE58DF31BD0345CE0DEF08
S11309B0BD04AEBD0A4B964091582208260F9641BD
S11309C091592309CE0DF9BD04AE7E02BBBD00FBD7
S11309D081F42308CE0E08BD04AE20629640913EF9
S11309E02208264A9641913F23447F003E7F003FE0
S11309F0CE0E11BD04AECE0E60BD04AED626D75BBE
S1130A009654109754BD02737F0026CE00B1861011
S1130A109730C604A6004625124624010C5A26F631
S1130A2046A700087A003026E920134620EFDE406E
S1130A30DF31CE003EBD08BBCE0E2FBD04AEDE407E
S1130A40DF31CE0058BD08BB7E02BB7F00407F0073
S1130A5041BD00F8812F23208D1F7D00272611C65C
S1130A60047800417900405A26F79B41974120E1E0
S1130A70CE0E3DBD00E920D9397F002781392203FC
S1130A80840F397C002739CE0E53BD04AECE006DE1
S1130A90C603BD00F8A100260D085A26F5CE0EA9FE
S1130AA0BD04AE7E0B59CE0EC2BD04AE7E02BB8623
S1130AB012913B22217D00682625BD00FB81B023D5
S1130AC0037C0068BD00FB81B022199621974796EC
S1130AD02297487E0757CE0EDBBD04AE7E02BBCE06
S1130AE00FC620F5BD00FB84079747BD00FB8407B4
S1130AF09748CE0EE6BD04AE20D97D0026260139E6
S1130B00BD00FB81B02230CE0069D62658BD055504
S1130B10DE69DF317D0057261FCE0058BD08BBBDFE
S1130B2004B3BD04B3DE69DF31BD0345CE0E71BD30
S1130B3000E9C6FABD0BE939CE003CBD08BBCE0EB8
S1130B40877E04AECE0F34BD04AE200DCE0F402000
S1130B50F6CE0F4ABD04AE2008CE0F79BD04AE20F8
S1130B6006CE0F8BBD04AECE0FF1BD04AEBD00F8B2
S1130B70814E27037E01007EE0E3DE6BA600905BDE
S1130B80D65C585858107D005D270B84BFC60AD721
S1130B9021D7227F004EA7004F975B975C975D3962
S1130BA0CE0061C6066D0027026A00085A26F6398F
S1130BB0BD00FB840716BD00FB8407D75ACE007125
S1130BC07C0020BD04D4E600C407965410975486D4
S1130BD080A700CE0FAFBD04AE9656BD025DBD0228
S1130BE0AD965ABD025D7E02BBCE0061BD00FB1115
S1130BF0230ABD00FB84030DA900A700088C00672D
S1130C0026EA7D006627037F005739CE0FC6BD0450
S1130C10AE7E02BBCE0FCEBD04AECE0FD9DF33CE37
S1130C2000616D002721DF5EDE33BD04AE08DF33D3
S1130C30DE5EC603BD00F25A26FAA600BD027508A0
S1130C408C006726DD20CADF5EDE3308080808DF73
S1130C5033DE5E20EA0A535041434520564F594142
S1130C6047452056332E32040A53204F52204C3F1E
S1130C702004205550040A4241534520494E205136
S1130C8004444F434B45440420444E0454554245C8
S1130C905320454D505459040A0A444154453A20BE
S1130CA0044B4C494E474F4E533A20045945415248
S1130CB0533A20045155414452414E543A2004536E
S1130CC04543544F523A20040A434F4D4D414E443C
S1130CD03A2004534849454C445320444F574E212D
S1130CE004534849454C445320555004434F5552EE
S1130CF053453A20045741525020464143544F52E1
S1130D003A2004424C4F434B454420415420530461
S1130D1052414D4D4544204B4C494E474F4E204186
S1130D205420530447414C415859204C494D49548F
S1130D3004544F525045444F2048495420044F55C1
S1130D4054204F4620454E45524759042020532EE7
S1130D50444154453A20042020434E44544E3A2002
S1130D600459454C4C4F5704524544044752454599
S1130D704E042020515544524E543A20042020530E
S1130D804543544F523A20042020454E455247597A
S1130D903A200420204B4C494E474F4E533A2004EE
S1130DA0202053484C44533A20042020544F52509E
S1130DB045444F3A20040D0A00000000040A53433E
S1130DC0414E20464F522051044D555354204C4F10
S1130DD057455220534849454C445304454E4552C7
S1130DE0475920415641494C41424C453A2004451B
S1130DF04E45524759203D2004454E4552475920FF
S1130E00544F4F204C4F57044D49534649524521A6
S1130E1004414C4C204C4F43414C204B4C494E47D1
S1130E204F4E532044455354524F59454421044591
S1130E304E454D592044414D4147454404203F20EF
S1130E4004535441520442415345044B4C494E47C8
S1130E504F4E040A50415353574F52442E2E2004F0
S1130E604B4C494E474F4E53204C454654203D2051
S1130E700420554E4954532048495420454E544566
S1130E80525052495345040A4B4C494E474F4E5316
S1130E902041545441434B3A20534849454C445310
S1130EA020484F4C44494E4704454E5445525052F5
S1130EB049534520444953494E54454752415445AA
S1130EC0530453455155454E43452041424F5254D6
S1130ED03A2050415353574F524404544F4F2045E6
S1130EE041524C5921044D414C46554E4354494FAF
S1130EF04E21040A0753504143452053544F524D49
S1130F003A20534849454C44532044414D414745B8
S1130F104421040A07534849502049532046524962
S1130F20454420464F522033524420415454454DA9
S1130F305054210407454E45524759203D20300462
S1130F400754494D4520555021040A07434F4E4745
S1130F50524154554C4154494F4E53210D0A0000FF
S1130F600000414C4C204B4C494E474F4E532044BB
S1130F70455354524F594544044D495353494F4ED8
S1130F802041204641494C55524504544845204689
S1130F90454445524154494F4E20495320534156EC
S1130FA04544210453555045524E4F564121040A9D
S1130FB00753555045524E4F564120494E20510437
S1130FC04241444C592044414D41474544040A445C
S1130FD0455620205354415404454E47045352531C
S1130FE0044C525304504853045452500453484C34
S1120FF0040A504C415920414741494E3F2004C7
S113A04AF7A070C608B6A074484848B8A07448482F
S113A05A79A07179A07279A07379A0745A26E6F668
S109A06AA070B6A07139DC
S105A048010011
S9030000FC
